:1016000012C021C020C01FC01EC01DC01CC01BC0F6
:101610001AC019C018C017C016C015C014C013C016
:1016200012C011C010C011241FBECFE5D4E0DEBF30
:10163000CDBF23E0A0E6B0E001C01D92AC33B207FD
:10164000E1F7B5D342C4DCCFE0E0F0E009950895BE
:101650001F93CF93DF93EC01162F17D4612FCE0188
:10166000939513D41FBA1EBADF91CF911F9108959D
:101670000F931F93CF93DF93EC018B0113D4B80129
:10168000CE0193950FD41FBA1EBADF91CF911F914F
:101690000F910895899AA29AB99A0895809130037A
:1016A0008F5F8093300390911502911105C080FDEA
:1016B00002C0C19A01C0C19880911502813009F41D
:1016C000C19A809130038A3078F010923003809173
:1016D0001502811105C080913B038A3028F401C0B6
:1016E00080E08F5F80933B030895CF93DF93109248
:1016F0001B0210926300C1E0D0E0CE01B9D39091FB
:101700001B02980F90931B0290916300892780938E
:1017100063002196CB30D10581F71FBA1EBADF9145
:10172000CF910895CF93DF9310921B021092630024
:10173000C1E0D1E0CE019CD390911B02980F909311
:101740001B02909163008927809363002196CB3020
:1017500081E0D80779F71FBA1EBADF91CF910895BB
:10176000CF93DF9310921B0210926300C1E0D0E090
:10177000CE017ED360911B02680F60931B02909193
:1017800063008927809363002196CB30D10581F7D0
:101790008EE090E07AD3609163008FE090E075D3A3
:1017A00060911B028EE091E070D3609163008FE046
:1017B00091E06BD31FBA1EBADF91CF910895E091EB
:1017C000600080912D03E81758F45D9903C0A89537
:1017D0005D9BFDCFF0E0EF5FFD4F80818CB901C0D4
:1017E000AA98809160008F5F8093600008959CB1FB
:1017F00080912C03811156C008B600FE08C080916C
:101800001A02813009F04BC010921A0204C0809174
:101810001A0281110FC09A32E9F588B7816088BF3A
:1018200012BE10922B038AE280932A0381E08093F8
:101830001A020895813071F580912B038F5F809398
:101840002B038D3810F010921A02E82FF0E0E859BF
:10185000FE4F908320912A03392F320F30932A03B1
:10186000833041F434E0390F3093FE013D3810F0FD
:1018700010921A023091FE0183130CC020932A03A8
:10188000921308C080911A02813021F480932C03B6
:1018900010921A0288B7816088BF12BE0895811124
:1018A000F9CFB9CF08952091040244E0420F85E0BA
:1018B000820F80932D03442369F0E1E0F2E02D5F75
:1018C00030E02E5F3D4F80E09191890FE217F307E2
:1018D000D9F701C080E0E42FF0E0EF5FFD4F808397
:1018E00081E080936000AA9A83E397E00197F1F783
:1018F0005D9903C0A8955D9BFDCF809101028CB9D5
:101900000895CF92DF92EF92FF92CF93DF93809171
:101910001C0290911D02A0911E02B0911F028093A3
:10192000310390933203A0933303B0933403409177
:1019300016025091170260911802709119028417D3
:101940009507A607B707B9F1C0903503D0903603C5
:10195000E0903703F0903803C4E6D0E0E0E2F2E034
:1019600040E050E09A01ABEABAEA76D296958795C4
:101970009C01220F331F820F931F4817590721F034
:101980008081841B8F5F04C080819EEF940F890F3C
:10199000C80ED11CE11CF11C89934F5F5F4F31963B
:1019A00040345105F9F6C0923503D0923603E092E7
:1019B0003703F0923803DF91CF91FF90EF90DF90E3
:1019C000CF900895A89561E081E090E041DE60E06D
:1019D00070E084E090E04CDE60E070E086E090E053
:1019E00047DE60E070E088E090E042DE6EEF8AE083
:1019F00090E02EDEA895B4DE089585E0A895C19A02
:101A00002FEF3FE191E0215030409040E1F700C0DE
:101A10000000C1982FEF3FE191E02150304090400D
:101A2000E1F700C00000815049F708951F93CF935C
:101A3000DF9381E090E01CD2813031F081E091E0D1
:101A400017D2813009F0BEDFA8958EE090E010D269
:101A5000C82F8FE090E00CD2D82F47DE80911B0278
:101A6000C81307C0C1E0809163008D1719F0C0E072
:101A700001C0C0E0A8958EE091E0FAD1D82F8FE0A8
:101A800091E0F6D1182F4EDE80911B02D81304C0CE
:101A900080916300181711F1CC2349F122C0A89559
:101AA000C1E0D0E0A895CE019395E2D1682FCE0198
:101AB000ECD12196CB30D105A9F752DE9EDF24C0B0
:101AC000A895CE01D5D1682FCE019395DED1219670
:101AD000CB30D105A9F744DE90DF16C0CC23F9F254
:101AE00013C0C13089F4A895C1E0D0E0E9CF6ADF26
:101AF00084DFA8952FEF8FE39BE02150804090403A
:101B0000E1F700C0000079DFDF91CF911F910895C8
:101B1000CF92DF92EF92FF921F93CF93DF93C0910A
:101B20006A0180910002C8133AC1E8E6F1E0118130
:101B3000D481D130A1F580916D01813031F5809350
:101B40001502E1E0F2E09AE29083C18312839CE007
:101B50009383848385838CE090E09783868381E000
:101B600092E09187808780912E0390912F03938735
:101B700082878091390390913A039587848780E426
:101B800090E0978786878FDE0AC110921502823017
:101B900009F052C08EEF80936C0180E019C0D23002
:101BA000B1F480911502813009F09BC060916D0104
:101BB0008EEF860F8D3F08F096C0609300028AE09A
:101BC00090E046DDCDDD1092150281E001C080E09D
:101BD00090916C01933089F590911502913009F044
:101BE000B0C0E8E6F1E0668170E0762F6627858177
:101BF000680F711D70932F0360932E0388E090E0AF
:101C000037DD6FEF83E090E023DDAADD109235032E
:101C100010923603109237031092380380E090E060
:101C2000A0E0BFEF8093160290931702A0931802D2
:101C3000B093190281E001C080E090916C01953071
:101C400009F054C090911502913009F09BC0809129
:101C50006D0190916E01A0916F01B0917001809320
:101C60001C0290931D02A0931E02B0931F02E3E793
:101C7000F1E0A0E2B2E023EB31E081918D932E17E9
:101C80003F07D9F73EDE60913103709132038091B6
:101C900033039091340361152BE0720781059105A0
:101CA00020F5C0901602D0901702E0901802F09034
:101CB00019026C157D058E059F0509F025D18091CF
:101CC000310390913203A0913303B0913403809398
:101CD000160290931702A0931802B093190281E0A4
:101CE00005C080E003C080E001C080E090916C01FD
:101CF000993039F590911502913009F043C0C090A8
:101D00006D01D0906E01E0906F01F09070014091F4
:101D1000350350913603609137037091380381E0A9
:101D2000C416D506E606F70609F080E0C416D50607
:101D3000E606F70639F561E083E090E089DC10DD26
:101D400081E090916C019E3FE9F4E1E0F2E08AE2EB
:101D50008083C183128384E083838EEF84838CE04D
:101D6000858380912E0390912F039783868383E050
:101D700090E07ED0813021F010920802109207028C
:101D800092DD0DC0E1E0F2E09AE29083C18312831C
:101D900093E0938394E69483D583868384DDDF91F7
:101DA000CF911F91FF90EF90DF90CF900895A8956D
:101DB00088E19FE00FB6F894A89581BD0FBE91BD54
:101DC00010BC97E199B98AB965DC30DE84E090E017
:101DD00057D090933A038093390386E090E050D037
:101DE000909362008093610088E090E049D09093E6
:101DF0002F0380932E038AE090E03AD08093000274
:101E000084E083BF8BE08EBD80E09DE29BBD8ABDF8
:101E1000C8E0A89508B604FE04C088B7806188BFF2
:101E20003DDC5F99E4DC5E9B02C05E9AC8DC809179
:101E30002C03882319F06CDE10922C0380913B0355
:101E40008450843030F7C0933B0383E090E010D09F
:101E50008130F9F6F9DBDDCFA29FB001B39FC0015D
:101E6000A39F01D0B29F700D811D1124911D089573
:101E7000E199FECF9FBB8EBBE09A99278DB3089561
:101E8000A8E1B0E042E050E012C0262FE199FECF79
:101E90009FBB8EBB2DBB0FB6F894E29AE19A0FBEA2
:101EA00001960895F2DF272FF1CFDC01CB01FC0171
:101EB000E199FECF06C0FFBBEEBBE09A31960DB2B2
:0E1EC0000D9241505040B8F70895F894FFCFAE
:101F0000E0E0FBE009950895CF92DF92EF92FF9217
:101F1000CF93DF936B017C01A8956FB7E199FECF5A
:101F2000A60183E0F60180935700E89507B600FC10
:101F3000FDCFC4EAD0E0A4E6B0E031E04456504022
:101F4000FA01EA0FFB1F11968C91119790E0982FE0
:101F500088272C91820F911D0C0130935700E89532
:101F600011241296AC17BD0759F785E0F60180934E
:101F70005700E89507B600FCFDCF81E1809357003C
:101F8000E8956FBFDF91CF91FF90EF90DF90CF90FA
:021F90000895B2
:0400000300001600E3
:00000001FF
